:020000040000FA
:1000000080311228FF3FFF3F7E1480310B1F1028E4
:100010002100931C10282000931C10289831B52033
:100020007E100900803114288731FE278031EB00D3
:1000300069308400233085008730FE000030FF00E7
:10004000903100208031FC015F3084000030850059
:100050000C30FE000030FF00903100208031A030D5
:100060008400003085004830FE000030FF009031F1
:100070000020803120308400013085003330FE00C4
:100080000030FF00903100208031A030840001302A
:1000900085001E30FE000030FF00903100208031CE
:1000A00020308400023085004B30FE000030FF001D
:1000B000903100207E10200088317028033020000D
:1000C000AB002B08F10063089831DE208031213E1F
:1000D00086000130870001080319272C0330200017
:1000E000AB002B08F10063089831DE208031213EFF
:1000F000860001308700013081022100EC01EC0A0A
:1001000003302000AB002B08F10063089831DE209B
:100110008031213E8600013087000108031D272C15
:1001200003302000AB002B08F10063089831DE207B
:100130008031203E860001308700011DBD2805303A
:100140002000AB002B08F10063089831DE208031DD
:10015000213E860002308700811703302000AB006B
:100160002B08F10063089831DE208031203E8600A4
:100170000130870001112100CA0103302000AB00CB
:100180002B08F10063089831DE208031203E860084
:1001900001308700011CF52903302000AB002B083B
:1001A000F10063089831DE208031203E8600013066
:1001B0008700010C2000AC00AC0C2C0C0F39003A6D
:1001C000031DF2280330AB002B08F10063089831BF
:1001D000DE208031203E860001308700010887390B
:1001E000083869290330AB002B08F1006308983107
:1001F000DE208031203E860001308700010C200087
:10020000AC00AC0C2C0C0F39013A031D172903303C
:10021000AB002B08F10063089831DE208031203ECE
:1002200086000130870001088739103869290330BA
:10023000AB002B08F10063089831DE208031203EAE
:10024000860001308700010C2000AC00AC0C2C0CA7
:100250000F39023A031DB4290330AB002B08F1001B
:1002600063089831DE208031223E8600013087000D
:10027000010803194A2903302000AB002B08F100C4
:1002800063089831DE208031203E860001308700EF
:10029000811CF52903302000AB002B08F100630816
:1002A0009831DE208031203E860001308700811C9D
:1002B0006B2903302000AB002B08F1006308983154
:1002C000DE208031203E860001308700010887391A
:1002D00018388100F52920006308AB00AC012B0819
:1002E000F1002C08F2000930F3000030F4009931DD
:1002F000882180316C302000AD002330AE007108C1
:100300002D07860072082E3D8700811D9629053035
:10031000AB002B08F10063089831DE208031233ECA
:1003200086000230870001030319F52903302000FD
:10033000AB002B08F10063089831DE208031203EAD
:100340008600013087008730810503302000AB0034
:100350002B08F10063089831DE208031203E8600B2
:10036000013087000110F5290330AB002B08F100A4
:1003700063089831DE208031203E860001308700FE
:10038000010C2000AC00AC0C2C0C0F39AD0003307C
:100390002D02031CF5290330AB002B08F100630884
:1003A0009831DE208031203E860001308700873082
:1003B000810503302000AB002B08F1006308983161
:1003C000DE208031203E860001308700011003309E
:1003D0002000AB002B08F10063089831DE2080314B
:1003E000203E86000130870081102100EC01272C7F
:1003F0000330AB002B08F10063089831DE20803118
:10040000203E860001308700011CBF2A03302000F7
:10041000AB002B08F10063089831DE208031203ECC
:10042000860001308700010C2000AC00AC0C2C0CC5
:100430000F39003A031D302A63089B31E6238031CF
:1004400003302000AB002B08F10063089831DE2058
:100450008031213E8600013087008101810ABB2A5C
:100460000330AB002B08F10063089831DE208031A7
:10047000203E860001308700010C2000AC00AC0C4F
:100480002C0C0F39013A031D692A63089B31B123F3
:10049000803104302000AB000330AC002C08F100A8
:1004A00063089831DE208031213E860001308700CC
:1004B00020002B0881000530AB002B08F1006308F9
:1004C0009831DE208031213E860002308700011401
:1004D000BB2A0330AB002B08F10063089831DE2003
:1004E0008031203E860001308700010C2000AC00E6
:1004F000AC0C2C0C0F39023A031D832A63089B3184
:10050000E6238031D32A0330AB002B08F1006308C7
:100510009831DE208031203E860001308700010CBA
:100520002000AC00AC0C2C0C0F39033A031DBB2A85
:1005300063089D312225803104302000AB00033058
:10054000AC002C08F10063089831DE208031213E98
:1005500086000130870020002B0881000530AB00A9
:100560002B08F10063089831DE208031213E86009F
:100570000230870081142100EC01EC0A272C0330A3
:100580002000AB002B08F10063089831DE20803199
:10059000203E860001308700011DE52A2000630807
:1005A0009E315926803104302000AB000330AC006E
:1005B0002C08F10063089831DE208031213E86004E
:1005C0000130870020002B08022C20006308AB00BC
:1005D000AC012B08F1002C08F2000930F3000030C8
:1005E000F4009931882180316A302000AD00233039
:1005F000AE0071082D07860072082E3D8700811914
:100600001F2B6308AB00AC012B08F1002C08F20093
:100610000930F3000030F4009931882180316C30CA
:100620002000AD002330AE0071082D07860072084F
:100630002E3D8700010E0F390139031D042C63087C
:10064000AB00AC012B08F1002C08F2000930F300DC
:100650000030F4009931882180316C302000AD00E9
:100660002330AE0071082D07860072082E3D8700EA
:10067000010E0F39023A031D852B6308963124269B
:10068000803120006308AB00AC012B08F1002C087E
:10069000F2000930F3000030F400993188218031F4
:1006A0006A302000AD002330AE0071082D078600AF
:1006B00072082E3D870001110330AB002B08F100BA
:1006C00063089831DE208031203E860001308700AB
:1006D0008730810503302000AB002B08F100630850
:1006E0009831DE208031203E8600013087000110E5
:1006F00003302000AB002B08F10063089831DE20A6
:100700008031203E86000130A22B630892316422A2
:10071000803120006308AB00AC012B08F1002C08ED
:10072000F2000930F3000030F40099318821803163
:100730006A302000AD002330AE0071082D0786001E
:1007400072082E3D8700811020006308AB00AC01C9
:100750002B08F1002C08F2000930F3000030F400FF
:100760009931882180316C302000AD002330AE00FB
:1007700071082D07860072082E3D8700010E0F3983
:10078000003A031DE02B6308AB00AC012B08F1001D
:100790002C08F2000930F3000030F4009931882170
:1007A00080316C302000AD002330AE0071082D0781
:1007B000860072082E3D870001080F395038022C40
:1007C0006308AB00AC012B08F1002C08F2000930E3
:1007D000F3000030F4009931882180316C30200022
:1007E000AD002330AE0071082D07860072082E3D43
:1007F0008700010E0F39AF00AF03AF0E01082F06BF
:100800000F392F068100BB2A6308AB00AC012B080F
:10081000F1002C08F2000930F3000030F4009931A7
:10082000882180316C302000AD002330AE0071088B
:100830002D07860072082E3D8700010E0F39AF008C
:10084000AF03AF0E01082F060F392F0681002100DC
:100850006C08031D312C943170248031013A031946
:10086000F82921006C08031D08009831C2200800F7
:10087000C4000530B6003608F10044089831DE2087
:100880008431203E8600023087003F3084000030F3
:10089000850005302000B70016001A00B70B4C2C5D
:1008A0004435A03E860001308700403FBB00413FF9
:1008B000BC004408B600B7013608F1003708F20062
:1008C0000930F3000030F400993188218431693017
:1008D0002000B8002330B90071083807860072087C
:1008E000393D870045308400003085000930BA006A
:1008F00016001A00BA0B782CC001210026083F39D7
:100900002000B6003608BD002100281D8C2C403088
:100910002000B6003608BD07673020003D06031DE5
:100920009F2C21004308031D9F2C2000431421000D
:10093000C301C30A20004408B6003608DF002000C7
:10094000431CAA2C67303D060319AA2C2100C301C1
:10095000200043103E303D06031DB22C4203031D10
:10096000B22CC2014408B6003608F7003D089031A9
:1009700066208431013A031DC02C4610C016982E03
:10098000431CC52C20004610D22C2100261FCA2C47
:10099000A81FC22C3E3020003D060319420803194F
:1009A000C22C46143D08B6003608C50021002708B1
:1009B0002000B6000330B636890BDB2C470836061C
:1009C000E0393606C7002100271DE92C2000461615
:1009D000EB2C200046122100A71CF02C2000C6148E
:1009E0002100271CF52C2000461503302000B600FE
:1009F0003608F10044089831DE208431223E86001A
:100A00000130870001080319142D03302000B600BF
:100A10003608F10044089831DE208431223E8600F9
:100A200001308700013081022100A81F062EC0304E
:100A300029052000B60040303606031D7C2D03300A
:100A4000B6003608F10044089831DE208431203E9B
:100A500086000130870001187C2D2100420820000B
:100A6000B6000330B7003708F10044089831DE20A3
:100A70008431223E86000130870020003608810044
:100A8000210028363C392000B6003608BE0021007F
:100A90002808033920003E07B6003608BE004A3059
:100AA0008600003087003E0881000330B60036081B
:100AB000F10044089831DE208431203E8600013068
:100AC0008700011403302000B6003608F100440806
:100AD0009831DE208431203E86000130870081106D
:100AE00020003E089A31B0228431B6004B30860097
:100AF0000030870036088100C03021002905200021
:100B0000B60080303606031DC72D0330B600360808
:100B1000F10044089831DE208431203E8600013007
:100B200087008118912E0330210028052000B6008F
:100B30004D083606FC393606CD00210029083F391C
:100B40002000B6003608BE003C30B6003608F10082
:100B50002100280903399831DE20843120003E0726
:100B6000B7003708BE004C308600003087003E08D2
:100B700081000330B6003608F10044089831DE20C9
:100B80008431203E8600013087008114912E21009F
:100B90002908C039031D912E29083F392000B600CD
:100BA0003608BE002100261FDA2D40302000B60096
:100BB0003608BE0703302000B6003608F1004408AE
:100BC0009831DE208431203E8600013087000119F3
:100BD000912E21004A08031D912ECA01CA0A4930EC
:100BE00086000030870020003E0881000330B600F8
:100BF0003608F10044089831DE208431203E86001A
:100C00000130870001152000C017912EA81D0B2E62
:100C1000200048140D2E200048102100281E132EFD
:100C20002000C814152E2000C8102100281F1B2EDC
:100C3000200048151D2E20004811C81C212E21001F
:100C4000B9012100A81E272E2000C815292E20003A
:100C5000C8112100280803392000B600B60EB60DD1
:100C6000470836061F393606C7000330B600360877
:100C7000F10063089831DE208431203E8600013087
:100C80008700010C2000B700B70C370C0F39023A6F
:100C9000031D542E0330210028052000B6004D0806
:100CA0003606FC393606CD004D11C61C5F2E4D159B
:100CB0000F30C80547081F39003A0319C615461DED
:100CC000672E4D1548080F392038C800C615210079
:100CD000A91F8F2E20004408B6003608F700210017
:100CE00029083F39903166208431003A03197B2E60
:100CF0003B134016912E3B173F3021002905200061
:100D0000B6003B083606C0393606BB002100291F55
:100D10008C2E2000BB17912E2000BB13912E20009B
:100D20003B132000431C982E5F0897311027843115
:100D30003F3086000030870005302000B6003608BE
:100D4000F10044089831DE208431203E84000230D6
:100D5000850005302000B70016001A00B70BAC2E36
:100D600045308600003087004408B600B7013608D9
:100D7000F1003708F2000930F3000030F400993137
:100D80008821843169302000B8002330B90071080F
:100D9000380784007208393D85000930BA00160012
:100DA0001A00BA0BCF2E4435A03E860001308700D2
:100DB0003B08C03F3C08C13F0800D900D301D30A1B
:100DC0000430CF004F08A000A101A10A0530D000D7
:100DD0005008F10059089831DE208631203E860007
:100DE000023087000108883107208631003A031954
:100DF000182F59088431382486310530CF004F0828
:100E0000F10059089831DE208631203E86000230FC
:100E10008700543084000030850005302000D00069
:100E200016001A00D00B102FF130D6055614DD2F06
:100E30000530CF004F08F10059089831DE20863187
:100E4000203E860002308700543084000030850048
:100E500005302000D00016001A00D00B2B2F5908A7
:100E6000CF00D0014F08F1005008F2000930F30024
:100E70000030F4009931882186316A302000D10099
:100E80002330D2007108510786007208523D870056
:100E900001100330CF004F08F10059089831DE20CF
:100EA0008631203E8600013087000110200059085D
:100EB000CF00D0014F08F1005008F2000930F300D4
:100EC0000030F4009931882186316D302000D10046
:100ED0002330D2007108510786007208523D870006
:100EE00081010330CF004F08F10059089831DE200E
:100EF0008631213E86000130870081012000560C9A
:100F00000739CF00CF0ACF0D56084F06F1394F06EB
:100F1000D600560C0739CF0003304F02031CDB2FDD
:100F200056106330CF004F08D400581C9A2F581029
:100F30002100C30120005908CF00D0014F08F10063
:100F40005008F2000930F3000030F4009931882194
:100F500086316A302000D1002330D2007108510759
:100F600086007208523D87000110210068080319AD
:100F7000DB2F200068080739063A031DC82F06300A
:100F8000CF004F08A90059088C312A248631DB2F65
:100F900068080739023A031DD62F0230CF004F08E8
:100FA000A90059088C312A248631DB2FF201013047
:100FB0009D31B92586312000D301543086000030A0
:100FC00087000530CF004F08F10059089831DE2026
:100FD0008631203E84000230850005302000D0009C
:100FE00016001A00D00BF02F5308080021008C15B2
:100FF0000430890BF92F21000C1608000234FF3F42
:101000007A30210099009801220096010800200002
:10101000A400A5012108A2002208F70024089931A4
:101020002A218831013A031D65282000A501A50A5F
:10103000A6012008260203185B28210803194C2862
:1010400099314021883120002008FF3EA200FF3066
:1010500003180030A300260822062304031D3F289E
:1010600001309C315D2488312000A2002608A63E74
:10107000860087012208810021000C1255280030CB
:101080009C315D2488312000A2002608A63E8600FF
:10109000870122088100552826084D3E8600013030
:1010A000870001089B317C23883101302000A20099
:1010B0002208A60719283230A20022082100CD00FC
:1010C0001230890B612800326B2801302000A20009
:1010D00022082100CE078731F627200025080800C6
:1010E0002200D5019831A92088319C31DE24883135
:1010F0000430DD005D08FA00103090310C2088319A
:10110000F20101309D31B92588319831652088314F
:10111000210068080319A12807302000DE001730DD
:10112000DD006A30890B9228DD0B9228DE0B9228B5
:1011300000002000A901A90A00308C312A2488313E
:10114000B12820006808F8390138E8006808DD0097
:101150005D08F70002309931A32188312100C801D0
:10116000C80A19302000DE005A30DD00B130890B8A
:10117000B728DD0BB728DE0BB72800320830200077
:10118000DD005D082200D60056089A3151228831D0
:1011900008302000DD005D082200D60739305602F5
:1011A000031CC42843302000DD005D082200D70066
:1011B00057089131D121883101302000DD005D08D0
:1011C0002200D70747305702031CD82821004F08B8
:1011D000031DF928280015082000DD000130DD3549
:1011E000FF3E031DEF285D35FC39DE005E0821005F
:1011F000CF008B170B174B302000DD005D0821005E
:10120000BE00CC0153080319022964002100D60155
:10121000200060089C319D2488312000DD005D089D
:10122000E0006B0803192B296008913156218831A1
:1012300021006803031D2D29200068080739023AA0
:10124000031D2D290330DD005D08A90060088C31E5
:101250002A2488312D29E301E001083020006406AA
:10126000031D4829393021006B02031C3D29083039
:101270002000DD005D082100EB006B089A3151224F
:10128000883108302000DD005D082100EB07C62909
:101290000C306406031D6B290230DD005D0821005F
:1012A000E10047306A02031C602943302000DD0062
:1012B0005D082100EA0041309131D1218831C629F1
:1012C0006A089131D121883101302000DD005D08AC
:1012D0002100EA07C62910306406031D73299531E1
:1012E00047258831C62902306B020318E718C62942
:1012F0006008DD005D082200D400200060089C31F9
:101300009D2488312000DD005D08E0000530DD000F
:101310005D08F10060089831DE208831233E8600A8
:101320000230870005300106031DAF29053020007B
:10133000DD005D08F100220054089831DE2088317C
:10134000233E86000230870005300106031DAF29C9
:10135000220054082000DD005D08E000C6292000BE
:10136000600891315621883121006803031DC62988
:10137000200068080739023A031DC6290330DD0042
:101380005D08A90060088C312A24883121006D0392
:10139000031DD029EC0180315E208831D601D60AA8
:1013A00022008D142100D301200064082100400296
:1013B0000318F3292000E40199316F2188312000BE
:1013C000DD005D082100E9000A3022005502031CFF
:1013D000ED29D5012100C609F32901302000DD00E7
:1013E0005D082200D5072100680803190229480872
:1013F000031D3B2A20006B0803193B2A06306402B8
:10140000031C042A5E30052A2130DD005D0821001E
:10141000B60022005508031D1E2AF20101309D313D
:10142000B925883101302000DD005D082200D50794
:1014300001302000DD005D082200D50721004308AF
:10144000031D262A200068080739312A04302000AD
:10145000DD005D08A9005F088C312A24883107303F
:101460002000DD005D08A90063088C312A24883142
:101470002100C701022921004708031D0229F201AA
:1014800001309D31B9258831C701C70A02292800DA
:1014900095010130F00070082100D807702B480337
:1014A000031D542A22008D159A31E2228A3121002F
:1014B000D401D40A07303F02031808003F0803197B
:1014C00008003F085802063EF0007008D8000800E7
:1014D000983174208A3121004803031D080022003E
:1014E0008D1108009A31E22208005D08031D7B2A55
:1014F000983174208A3120006208031D0800210001
:101500006C03031D882A5E30F0007008E0000800BC
:101510003F30F0007008E0000800983174200800A7
:101520009A31E2228A3120006208031D080021005E
:101530005603031DBC2A6F08F00070082000E60067
:101540007C08F0007008E50021006E08F0007008CB
:10155000DC005E08F0007008DB0020006608F00088
:1015600070082100DA0020006508F00070082100F2
:10157000D9002100ED0108005A08F0007008200091
:10158000E60021005908F00070082000E50008007E
:101590002000E61B08008D2A9C311D240800200035
:1015A000661B08008D2A2000E61A08008D2A2000FC
:1015B000661A08008D2A2000E61908008D2A2000EE
:1015C000661908008D2A2000E61808008D2A2000E0
:1015D000661808008D2A2000E51B08008D2A2000CF
:1015E000651B08008D2A2000E51A08008D2A2000BE
:1015F000651A08008D2A2000E51908008D2A2000B0
:10160000651908008D2A983187208A31013A031D17
:101610000D2B22000D138D13080022008D130800DE
:10162000983187208A31013A031D1A2B22000D13AD
:101630008D12080022000D1308009C311D248A31F0
:1016400020006203031D392B0130F0007008E4070D
:101650002100D401D301D30AED01ED0A3E08280090
:1016600096001F30970021003A08F0007008E10052
:1016700008000230280095002000E201E20A210063
:101680005C08F00070082000E60021005B08F00014
:1016900070082000E500671C532B0930F00070082B
:1016A0002100D80008000830F00070082100D800A0
:1016B0000800410828009600063097002100D80154
:1016C0002000E2012100ED01ED0A08004108280098
:1016D0009600063097002100D8012000E201B92AC7
:1016E0005808013A03194F2A033A0319292C013AE1
:1016F0000319292C073A0319292C013A0319292C1B
:10170000033A0319292C013A0319292C0F3A03191A
:10171000292C013A0319682A033A0319722A013A5B
:101720000319752A073A03198D2A013A0319902AD9
:10173000033A0319C82A013A0319CC2A1F3A03199C
:10174000722A013A0319CF2A033A0319CC2A013A23
:101750000319722A073A0319D32A013A0319CC2A2A
:10176000033A0319722A013A0319D72A0F3A0319C7
:10177000CC2A013A0319722A033A0319DB2A013AE7
:101780000319CC2A073A0319722A013A0319DF2AEE
:10179000033A0319CC2A013A0319722A3F3A031972
:1017A000E32A013A0319CC2A033A0319722A013AAF
:1017B0000319E72A073A0319CC2A013A0319722AB6
:1017C000033A0319EB2A013A0319CC2A0F3A0319F9
:1017D000722A013A0319EF2A033A0319CC2A013A73
:1017E0000319722A073A0319F32A013A0319CC2A7A
:1017F000033A0319722A013A0319F72A1F3A031907
:10180000CC2A013A0319722A033A0319FB2A013A36
:101810000319CC2A073A0319722A013A0319FF2A3D
:10182000033A0319CC2A013A0319722A0F3A031911
:10183000032B013A0319CC2A033A0319722A013AFD
:101840000319102B073A03191D2B013A0319592BC1
:10185000662B0800CD000530AA002A08F1004D08CB
:101860009831DE208C31203E8600023087004430E3
:1018700084000030850005302000AB0016001A00FF
:10188000AB0B3E2C4D08AA00AB012A08F1002B0837
:10189000F2000930F3000030F400993188218C31D6
:1018A00003302000AA002A08F1004D089831DE20FC
:1018B0008C31203E860001308700403F2000C1006F
:1018C000413FC200423FC300F20193309D31B92530
:1018D0008C31F201F20A36089D31B9258C31E42FA2
:1018E000F20101309D31B9258C31F201C5309D31B5
:1018F000B9258C3100302000A0009830A1000A30BA
:10190000AA002A08A2009A3128228C31F2019B30C9
:101910009D31B9258C310A302000A0009830A100FB
:101920000330AA002A08A2009A3128228C31F20141
:10193000F20A34309D31B9258C31F201F20A0130BE
:1019400098319D208C31083E9D31B9250800063024
:1019500021006902031CB32C46080319B32C200094
:101960004D08FA3EB52C20004D08AA002A08C000F8
:1019700006304002031808000330AA002A08F100CC
:1019800040089831DE208C31013E2000AB002B084E
:10199000CC004D08AA00AB012A08F1002B08F20088
:1019A0000930F3000030F400993188218C3169301E
:1019B0002000AC002330AD0071082C0786007208AF
:1019C0002D3D87000108AE00AF012E08C9002F0889
:1019D000CA0000304A023E3003194902031CF62CAB
:1019E0004908FD3EC900FF304A3DCA004D08AA0023
:1019F000AB012A08F1002B08F2000930F300003097
:101A0000F400993188218C3171302000AC002330F2
:101A1000AD0071082C07860072082D3D87004A082A
:101A2000A3004908A2000230AA002A08A4004C081A
:101A3000AB002B08A5000230AC002C08A6002E300D
:101A4000AD002D08A7009E31AF268C312100EF1B81
:101A5000562D7C082000AA000330AA36890B2D2DB4
:101A60002A08AB00AC012B08C9002C08CA007C1D59
:101A70003B2D7F303C2D7E30AA002A08CB004A083F
:101A8000A3004908A2000330AA002A08A4004C08B9
:101A9000AB002B08A5000230AC002C08A6004B08B8
:101AA000AD002D08A7009E31AF260800F2012000EE
:101AB0004C08D33E9D31B9258C312000E71E5C2EA9
:101AC000440821003B06031D080020004408AA002A
:101AD0002A08CC0031304C020318782D4C08AA009B
:101AE0000330AA36890B712D2A08AB002B08CC00D5
:101AF0004C08AA00AB012A08A2002B08A30004305E
:101B0000AC002C08A400A501A50A0230AD002D08E8
:101B1000A6002030AE002E08A7009E31AF268C31E3
:101B200020004D08AA00AB012A08F1002B08F200A2
:101B30000930F3000030F400993188218C316F3086
:101B40002000AC002330AD0071082C07860072081D
:101B50002D3D87000108AE00AF012E08BE002F0802
:101B6000BF003F08A3003E08A2000430AA002A08D4
:101B7000A4000430AB002B08A5000230AC002C08F8
:101B8000A6002030AD002D08A7009E31AF268C3175
:101B900020004D08AA00AB012A08F1002B08F20032
:101BA0000930F3000030F400993188218C31703015
:101BB0002000AC002330AD0071082C0786007208AD
:101BC0002D3D87000108AE00AF012E08BE002F0892
:101BD000BF003F08A3003E08A2000430AA002A0864
:101BE000A4000730AB002B08A5000330AC002C0884
:101BF000A6002030AD002D08A7009E31AF268C3105
:101C000020004D08AA00AB012A08F1002B08F200C1
:101C10000930F3000030F400993188218C316D30A7
:101C20002000AC002330AD0071082C07860072083C
:101C30002D3D87000108AE002E08CC003E304C023E
:101C4000031C242E0330CC024C08AA00AB012A0846
:101C5000A2002B08A3000430AC002C08A4000B3019
:101C6000AD002D08A5000330AE002E08A6002030E0
:101C7000AF002F08A7009E31AF268C31F201F20A87
:101C8000200041080139303E9D31B9258C31F201E7
:101C9000F20A2000410C0139303E9D31B9258C31CA
:101CA000F201F20A2000410CAA00AA0C2A0C0F39FA
:101CB000413E9D31B9250800671E7B2EF201F20AD4
:101CC00041080139303E9D31B9258C31F201F20ACB
:101CD0002000410C0139303E9D31B9258C31F20193
:101CE000F20A2000410CAA00AA0C2A0C0F39413E2E
:101CF0009D31B92508007C1E7F2E4630802E2D3068
:101D0000AA002A08CB00F201F20A4B089D31B9253E
:101D10008C31FC1E8D2E46308E2E2D302000AA00D8
:101D20002A08CB00F201F20A4B089D31B9258C310B
:101D30007C082000AA000230AA36890B9C2E2A08B3
:101D40000339343CAB002B08CB00F201F20A4B08FC
:101D50009D31B9250800063021006902031CB72E09
:101D600046080319B72E20004D08FA3EB92E200070
:101D70004D08AA002A08C0000630400203180800D7
:101D80000330AA002A08F10040089831DE208C3187
:101D9000013E2000AB002B08CC004708613EAA00A2
:101DA0002A08CB004408AA00AB012A08C9002B0866
:101DB000CA00633049064A04031DE32E7830AA00A6
:101DC0002A08CB00F52E023047020318F52E4A08E8
:101DD000AB004908AA00AB36AA0CAB36AA0CAB364E
:101DE000AA0C2A08C9002B08CA004A08A3004908FF
:101DF000A200A401A40A4C08AA002A08A5000230E7
:101E0000AB002B08A6004B08AC002C08A7009E31A5
:101E1000AF26080021004308031908002000481CD1
:101E200008005F08AA00AB012A08F1002B08F200A5
:101E30000930F3000030F400993188218C316F3083
:101E40002000AC002330AD0071082C07860072081A
:101E50002D3D87000108AE00AF012E08BE002F08FF
:101E6000BF003F08A3003E08A2000430AA002A08D1
:101E7000A4000F30AB002B08A5000230AC002C08EA
:101E8000A6002030AD002D08A7009E31AF268C3172
:101E900020005F08AA00AB012A08F1002B08F2001D
:101EA0000930F3000030F400993188218C31703012
:101EB0002000AC002330AD0071082C0786007208AA
:101EC0002D3D87000108AE00AF012E08BE002F088F
:101ED000BF003F08A3003E08A2000430AA002A0861
:101EE000A4001230AB002B08A5000330AC002C0876
:101EF000A600A7019E31AF260800BC01BC0A06302F
:101F00003C020318AF2F3C0898319D208C312000F3
:101F1000AA00AB012A08A2002B08A3000230AC00E3
:101F20002C08A4003C08AD000130AD35FF3E031D78
:101F3000952F2D35FD3EAE002E08A5000330AF00D5
:101F40002F08A6002030B0003008A7009E31AF2631
:101F50008C3101302000AA002A08BC077F2F1430E2
:101F6000AA002A08BD001B303D02031808003D08E6
:101F700098319D208C312000AA00AB012A08A200D4
:101F80002B08A3000330AC002C08A4000330AD00E4
:101F90002D08F1003D089831DE208C31C53E20002F
:101FA000AE002E08A5000230AF002F08A60020309A
:101FB000B0003008A7009E31AF268C3101302000E0
:101FC000AA002A08BD07B32F20002908013A0319E7
:101FD000702C033A0319A72C013A0319AB2E073AC8
:101FE00003190A2F013A0319FF2F033A0319FF2F90
:101FF000013A03197D2F0E3A0319FF2FFF2F080016
:102000006400800101310130FE020030FF3B7F0897
:102010007E040319003401286830FB00E430890B8A
:102020000F28FB0B0F280032F20130309D31B9250B
:1020300090312030FB002A30890B1C28FB0B1C2818
:10204000F20130309D31B9259031A0300032890B3A
:102050002628F20130309D31B9259031A030003270
:10206000890B2F28F20120309D31B92590317A0358
:10207000031D3D28F2012430432804307A06031D55
:102080004628F20128309D31B9259031F2010C30FB
:102090009D31B9259031A0300032890B4C28F201D6
:1020A00001309D31B9259031A0300032890B55287F
:1020B000F20106309D31B9259031A0300032890BF4
:1020C0005E28F20140309D31B92508002000A100B2
:1020D000A001A201220877060319D3280530F800D1
:1020E0007808F10022089831DE209031223E8600E7
:1020F00002308700011CD32820002208F800F901D3
:102100007808F1007908F2000930F3000030F4009B
:102110009931882190316930FA002330FB00710831
:102120007A07860072087B3D87000108200021069F
:10213000031DBB282208F800F9017808F10079088E
:10214000F2000930F3000030F40099318821903119
:102150006A30FA002330FB0071087A0786007208A3
:102160007B3D8700011CBB282000A001A00A0E3087
:10217000F8007808A20020002235A03E8600013039
:10218000870001083F392106031DD3282235A03ED0
:10219000860001308700011FD328A001A00A0E305D
:1021A000F8007808A2000130F80078082000A207A3
:1021B0000E302202031C6A2820080800A000A1019A
:1021C0000530F8007808F10021089831DE209031C0
:1021D000223E86000230870001184C29200020088A
:1021E000F8000530F9007908F10021089831DE2067
:1021F0009031203E8600023087007808810005304B
:10220000F8007808F100200021089831DE20903194
:10221000223E86000230870001140530F80078085D
:10222000F100200021089831DE209031223E860006
:1022300002308700F13081057708F8000530F90099
:102240007908F100200021089831DE209031233EEA
:102250008600023087007808810020002108F800FD
:10226000F9017808F1007908F2000930F300003034
:10227000F4009931882190316A30FA002330FB0054
:1022800071087A07860072087B3D870001100E30C6
:10229000F80078082000A1000130F800780820003C
:1022A000A1070E30210203180800E028DC000430EA
:1022B000DA005A08CE005C088631DD269131013AF9
:1022C000031DCB290530DA005A08F1005C0898316B
:1022D000DE209131233E8600023087000530010662
:1022E000031D8F2903302000DA005A08F1005C0832
:1022F0009831DE209131203E860001308700011D9B
:102300008F2905302000DA005A08F1005C08983166
:10231000DE209131213E8600023087008117053092
:102320002000DA005A08F1005C089831DE20913173
:10233000213E86000230870001082000DB005B0898
:102340002200CD00983192209131003A0319AA2938
:102350002200CD152000A001A00AA1010530DA005D
:102360005A08F1005C089831DE209131203E860049
:102370000230870001088831072091310530DA00EA
:102380005A08F1005C089831DE20213E86000230B8
:102390008700810108000130DA005A082100CE07C9
:1023A00008002000A9005E2A41309A3102229131B2
:1023B000003A031908000430A7002708A000A10173
:1023C000A10A4130883107209131003A03190800F1
:1023D00021002608031D08000C3027052000A70057
:1023E0000C302706031D08004630A7002708F90017
:1023F00043309931E0219131A8002808E1006108BB
:1024000003191A2A61080739A7000330A735FF3ED0
:10241000031D062A2735063EA80028082200CD0005
:1024200002302000A7002708F70061089031DE2065
:1024300091311C2A2200CD012000A001A00AA10197
:1024400041308831072008002100CB0142309A3109
:1024500002229131003A031908004330A7002708EF
:10246000AA002A089A317F229131003A031D542A8A
:1024700006302000A7003030890B3C2AA70B3C2AED
:10248000000020002A089A3102229131003A0319F3
:10249000512A0230A7002708F7002A089031DE20D1
:1024A00091312100CB01CB0A01302000A700270881
:1024B000AA0747302A0203180800312A2908413A9E
:1024C0000319D429242A0800F9007908A500A601D7
:1024D0002508F1002608F2000930F3000030F4006E
:1024E0009931882192316B302000A7002330A80059
:1024F0007108270786007208283D870001081F39E8
:10250000A9000230A935FF3E031D822A2935AA0001
:102510002A08FC007935A03E860001308700011FA3
:10252000CC2A7935A13E8600013087000118CC2ADB
:102530007935A03E86000130870001083F39A500AB
:1025400025082100EF006F082000A50025082100C4
:10255000EE007935A13E860001308700011479082C
:102560002000A500A6012508F1002608F200093088
:10257000F3000030F4009931882192316C30200052
:10258000A7002330A8007108270786007208283D9D
:1025900087000F308105FE2AF70179089D316C25EF
:1025A000923179082000A500A6012508F10026082F
:1025B000F2000930F3000030F400993188219231A3
:1025C0006A302000A7002330A80071082707860082
:1025D0007208283D8700010E0139A9000130A93594
:1025E000FF3E031DEF2A29357C07AA002A08FC00BC
:1025F0007935A13E86000130870001107C08A500D6
:1026000025082100DE000800A0002008F700F801DE
:102610007708F1007808F2000930F3000030F40088
:102620009931882193316930F9002330FA0071081B
:102630007907860072087A3D8700213084000030D7
:1026400085000930FB0016001A00FB0B232B20002D
:10265000A10122100F30A405A801A601A501033095
:10266000F7007708F10020089831DE209331203EF2
:1026700086000130870001100330F7007708F10071
:10268000200020089831DE209331203E8600013062
:10269000870081100330F7007708F1002000200840
:1026A0009831DE209331203E86000130870087304C
:1026B00081050330F7007708F100200020089831E9
:1026C000DE209331203E8600013087000111033067
:1026D000F7007708F100200020089831DE209331C0
:1026E000213E86000130870081010330F700770822
:1026F000F100200020089831DE209331223E860030
:1027000001308700810121308600003087002000E1
:102710002008F700F8017708F1007808F200093086
:10272000F3000030F4009931882193316930F900C9
:102730002330FA0071087907840072087A3D850019
:102740000930FB0016001A00FB0BA22B0800023018
:1027500098319D2093312000A0002008E8006808EF
:102760000739003A031DB82B2100C801C80ABA2B4B
:102770002100C801033098319D2093312000A00032
:102780002008E700043098319D2093312000A000FC
:1027900020082100C200143098319D209331200080
:1027A000A00020082100C000153098319D209331F1
:1027B0002000A00020082100C100163098319D2083
:1027C000933107392000A00020082100BF000A3003
:1027D000F2000030F300173098319D209331053E10
:1027E000F400003003180130F5009E3108269331C3
:1027F00072082000A0002008EA000A30A00020088B
:10280000F1006A089831DE2093312000A1002108F0
:10281000EA0047306A02031C112C4630A000200851
:10282000EA006A08A0002008F70017309931A321B8
:1028300093310A30F2000030F300183098319D20B7
:102840009331053EF400003003180130F5009E314D
:102850000826933172082000A0002008E9000A3001
:10286000A0002008F10069089831DE209331200093
:10287000A1002108E90033306902031C432C3230E7
:10288000A0002008E9006908A0002008F70018301F
:102890009931A32193311A3098319D209331200032
:1028A000A00020082100BD00193098319D209331EF
:1028B0002000A00020082100BE003D083E020318B1
:1028C000672C3D082000A00020082100BE00053034
:1028D00098319D202000A00020082100BB000800A6
:1028E0002000A001A101210821006902031CE42CA1
:1028F00020002108F700F8017708F1007808F200BD
:102900000930F3000030F4009931882194316A30A5
:10291000F9002330FA0071087907860072087A3DC1
:102920008700811DDE2C20002108F700F8017708C0
:10293000F1007808F2000930F3000030F40099311A
:10294000882194316A30F9002330FA007108790740
:10295000860072087A3D8700811120002108F70067
:10296000F8017708F1007808F2000930F300003030
:10297000F4009931882194316A30F9002330FA004B
:1029800071087907860072087A3D8700011CDE2CE9
:1029900020002108F7007708E3000330F7007708EC
:1029A000F10063089831DE209431213E8600013029
:1029B00087008101810A2000A001A00A0130F700F0
:1029C00077082000A107732C20002008031D442D48
:1029D000630821006906031DF02C2000A101F62CDC
:1029E00020006308013EF7007708A1002108630674
:1029F0000319272D2108F700F8017708F10078085E
:102A0000F2000930F3000030F4009931882194314C
:102A10006A30F9002330FA007108790786007208DD
:102A20007A3D8700011C1C2D20002108F700770843
:102A3000E300A001A00AF62C210069082000210271
:102A40000318ED2C0130F7007708A107F62C2108B8
:102A5000F700F8017708F1007808F2000930F30078
:102A60000030F4009931882194316A30F900233024
:102A7000FA0071087907860072087A3D8700011C08
:102A8000442D2000A001A00A2000200808004830A2
:102A90009831CF209531013A031D08000430CE0053
:102AA0004E08A000A101A10A4830883107209531C5
:102AB000003A03190800D301D0015308A63E86004E
:102AC000870149300102031CBE2D5308A63E860033
:102AD00087014D3001020318BE2DD1015308A63ED7
:102AE000860087010530CE004E08F100510898316C
:102AF000DE209531203E840002308500000801066A
:102B0000031D992D05302000CE004E08F10051081C
:102B10009831DE209531223E860002308700011C6C
:102B2000992D2000D001D00A0E30CE004E08D100E1
:102B30009E2D01302000CE004E08D1070E305102EC
:102B4000031C6E2D5008031D1B2E0530CE004E08B1
:102B5000F7005308A63E8600870101089031DE2069
:102B600095315308A63E860087010108CE00530820
:102B7000A03E860087014E0881001B2E5308A03E10
:102B800086008701010803191B2ED2015308A03EBD
:102B9000860087010530CE004E08F10052089831BA
:102BA000DE209531203E84000230850000080106B9
:102BB000031D122E05302000CE004E08F1005208F1
:102BC0009831DE209531223E860002308700011CBC
:102BD000122E63302000CE000530CF004F08F100E8
:102BE00052089831DE209531203E86000230870061
:102BF00020004E0881000330CE004E08A900520884
:102C00008C312A24953120005308A03E860087018C
:102C100081015208933104239531200052089B31E1
:102C20001523953101302000CE004E08D2070E301A
:102C30005202031CC62D0130CE004E08D3070430CB
:102C40005302031808005C2DF9007908A500A601BD
:102C50002508F1002608F2000930F3000030F400E6
:102C60009931882196316B302000A7002330A800CD
:102C70007108270786007208283D8700010E890C1D
:102C80000739A9000130A935FF3E031D432E293520
:102C9000AA002A08FC007908A500A6012508F10071
:102CA0002608F2000930F3000030F4009931882141
:102CB00096316C302000A7002330A8007108270748
:102CC00086007208283D870001187C167908A50047
:102CD000A6012508F1002608F2000930F3000030B3
:102CE000F4009931882196316C302000A700233000
:102CF000A8007108270786007208283D8700811800
:102D0000FC167908A500A6012508F1002608F200A6
:102D10000930F3000030F4009931882196316C308D
:102D20002000A7002330A80071082707860072083A
:102D3000283D87000119FC177908A500A601250880
:102D4000F1002608F2000930F3000030F400993158
:102D5000882196316C302000A7002330A80071082C
:102D6000270786007208283D870081197C1779356E
:102D7000A03E860001308700011FFC2E7935A13E60
:102D80008600013087008118FC2E7935A03E860030
:102D90000130870001083F39803EA5002508210049
:102DA000EF006F082000A50025082100EE0079350E
:102DB000A13E860001308700811479082000A5001B
:102DC000A6012508F1002608F2000930F3000030C2
:102DD000F4009931882196316C302000A70023300F
:102DE000A8007108270786007208283D870001089F
:102DF0000F3940388100092F8030A5002508F700E1
:102E000079089D316C257935A13E86000130870017
:102E100081107C082000A50025082100DE000800A4
:102E2000B5003508A200A3012208F1002308F20032
:102E30000930F3000030F4009931882197310330D4
:102E40002000A2002208F10035089831DE209731D9
:102E5000203E860001308700011C0800033020005E
:102E6000A2002208F10035089831DE209731203E7B
:102E7000860001308700811C080021004508031DE1
:102E8000442FC501C50A080020003508A200A3018F
:102E90002208F1002308F2000930F3000030F400AA
:102EA0009931882197316F302000A4002330A5008C
:102EB0007108240786007208253D87000103031D61
:102EC0006B2FF701F70A08309931A32197319F3111
:102ED00017279731E22F3508A200A3012208F1003D
:102EE0002308F2000930F3000030F4009931882102
:102EF000973170302000A4002330A500710824070A
:102F000086007208253D87003508A600A70126081F
:102F1000F1002708F2000930F3000030F400993185
:102F2000882197316F302000A8002330A900710854
:102F3000280784007208293D8500000898319D20EB
:102F4000973101060319E22F20003508A200A301E2
:102F50002208F1002308F2000930F3000030F400E9
:102F600099318821973170302000A4002330A500CA
:102F70007108240786007208253D87000108A60015
:102F80002608F7003508A700A8012708F10028083F
:102F9000F2000930F3000030F400993188219731B4
:102FA0006F302000A9002330AA007108290786008D
:102FB00072082A3D870001089931A3219731933186
:102FC000A72397312100C50103302000A200220869
:102FD000F10035089831DE209731203E860001301F
:102FE0008700011003302000A2002208F1003508FC
:102FF0009831DE20203E86000130870081100800D5
:1030000043342D344434693467346934743461345E
:103010006C34003456342E340034FF3FFF3FFF3F02
:10302000FF3FFF3FFF3FFF3FFF3FFF3FFF3FFF3FB0
:10303000FF3FFF3FFF3FFF3FFF3FFF3FFF3FFF3FA0
:10304000FF3FFF3FFF3FFF3FFF3FFF3FFF3FFF3F90
:10305000FF3FFF3FFF3FFF3FFF3FFF3FFF3FFF3F80
:10306000FF3FFF3FFF3FFF3FFF3FFF3FFF3FFF3F70
:10307000FF3FFF3FFF3FFF3FFF3FFF3FFF3FFF3F60
:10308000FF3FFF3FFF3FFF3FFF3FFF3FFF3FFF3F50
:10309000FF3FFF3FFF3FFF3FFF3FFF3FFF3FFF3F40
:1030A000FF3FFF3FFF3FFF3FFF3FFF3FFF3FFF3F30
:1030B000FF3FFF3FFF3FFF3FFF3FFF3FFF3FFF3F20
:1030C000FF3FFF3FFF3FFF3FFF3F2800171508006E
:1030D000FB3021008C000800383021008C000800F3
:1030E000163021009700080022008D120D138D1359
:1030F000080072082200D9007108D80008002100D9
:103100000C120430890B822821008C110800200049
:103110000D1D8E282100B701B70A90282100B701A4
:103120003708080020008D1899282100C401C40A1E
:103130009B282100C40144080800F1007108230005
:1031400091001513951315140000000023001308B7
:103150000800993101219831883100209831983147
:10316000702098319831EF200800931028009501C5
:1031700021006108031DBF288A3147220800013061
:10318000E10208003E30F1007108EF00FC013E3022
:10319000F1007108EE00DE01EC01EC0A0800A1006C
:1031A000F701210899312A2198312000A000200838
:1031B000A2008731F627200022080800F400F3015E
:1031C000741CE6287108F2007208F3070310F10D71
:1031D0000310F40C7408031DE02873080800313054
:1031E00028009600950120009310210093140030D0
:1031F000F1000030F2009831792006302800970065
:1032000008008C018D01383021008C0016308D00B3
:1032100023008D018C01143024008D008C012100CD
:10322000951322009D019E0108003208303EF100F6
:103230007108E6003008303EF1007108E5002E0804
:10324000303EF1007108E4002C08303EF1007108B6
:10325000E3000800F90098317F209931793577072C
:10326000F8007808FA007A089B317C239931003AFB
:10327000031D3D29FB01FB0A3E29FB017B080800D9
:103280002100C901C90A8C15F20120008C1D4E29AC
:103290006030F1007108F2002100C9010130F10035
:1032A0007108F20760307202031808004529F10026
:1032B000711C5D2922008C145F2922008C10F11CE6
:1032C00063290C1464290C10711D68298C17692955
:1032D0008C13F11D6D290C1708000C1308000D301C
:1032E000F5007508F6000530F5007508F100760860
:1032F0009831DE209931223E860002308700011885
:1033000086290130F6027608031D73297608080025
:10331000F501F601711C90297308F5077408F63D54
:103320000130F335F40D890B91290130F236F10C9F
:10333000890B962971087204031D8A297608F20008
:103340007508F1000800F80078082300910077085C
:10335000930095131513151500308B1B0130F900E0
:103360008B1355309600AA30960095149518B629FF
:103370001511790C031C8B1303188B170800F1012E
:1033800098316820993122008D110D140C150530EB
:10339000890BC829000020000C1FD029F101F10A77
:1033A00022000C110530890BD329000022000C15D6
:1033B0000530890BD929000022000C117108080082
:1033C000A000A1012008FA007A08A20022087902D0
:1033D000031C002A22089A317F229931003A031DEA
:1033E000FA2920002208FA007A08A1007908FA00D8
:1033F0007A08A2000130FA007A082000A207E62924
:10340000210808002000A100A201F701210899313C
:103410002A219A31003A0319232A8D309B317C23CB
:103420009A31FF3A2000A0002008A2008731F62739
:103430009A3115302000A000C630890B1D2AA00B40
:103440001D2A0000252A8731F627200022080800BF
:10345000A3012208FF3EFA00FF3003180030FB00F2
:103460007B08803A803C031D372A7A082302031820
:103470000800F201F20A20002108FB002008FA00EF
:1034800023087A0784007B0803187B0A850000085C
:103490009D31B9259A310130FA007A082000A3073E
:1034A000292A2000A8002100CB01200028089A31F9
:1034B0007F229A31003A031D080004302000A70043
:1034C0002708A000A101A10A2808883107209A3105
:1034D000003A031908003F30210026052000A7000C
:1034E0003E302706031D792AF70128089031DE2097
:1034F0000800F701F70A28089031DE200800F600DE
:10350000F701F8010530F5007508F10078089831E9
:10351000DE209A31203E86000230870001087606C0
:10352000031DA62A0530F5007508F10078089831CA
:10353000DE209A31223E860002308700011CA62A36
:10354000F701F70A0E30F5007508F8000130F500B4
:103550007508F8070E307802031C822A77080800E5
:10356000F4007408F1000230F136890BB42A7108B6
:103570000739F2007208F50074080339F1000230CF
:10358000F135FF3E031DC02A71357507F200720840
:10359000F500740820397507F1007108F500750809
:1035A000F1000330F136890BD22A71080739090777
:1035B000F2007208F30075087307F1007108F50056
:1035C00075080800FB2A0D30890BE42A0000102B37
:1035D0001A30890BE92A0032102B2830890BEE2A89
:1035E000102B3530890BF22A0000102B4230890B4A
:1035F000F72A0032102B20006908003A0319102B1B
:103600000A3A0319E32A1E3A0319E82A0A3A031967
:10361000ED2A363A0319F12A1A3A0319F62A102B21
:1036200022008D160D178D170800A0000530F5003B
:103630007508F10020089831DE209B31203E86007D
:103640000230870021308400003085000530F6000C
:1036500016001A00F60B282B2000A1012310F130D0
:10366000A30521308600003087000530F50075087D
:10367000F10020089831DE209B31203E840002308A
:1036800085000530F60016001A00F60B432B0800E3
:10369000F701F801710872040319772BF601F60A95
:1036A000F21B5C2B0130F135F20D890B532B0130ED
:1036B000F5007508F607502B0130F735F80D890B2A
:1036C0005D2B72087402031D672B71087302031CC3
:1036D0006E2B7108F3027208F43B77140130F23656
:1036E000F10C890B6F2B0130F602031D5C2B78085F
:1036F000F2007708F1000800F50021000C12F60135
:10370000F51F842B0C16852B0C1200320032003270
:10371000003221008C157535F3007308F500013077
:10372000F3007308F6078C1108307602031C802B17
:103730000C160430890B9A2B21008C1599314021ED
:1037400021008C15003020000C1A0130F4002100FB
:103750008C11003200320032003221000C12740849
:103760000800F900C030A5002508F70079089D3150
:103770006C259B3179082000A500A6012508F100E1
:103780002608F2000930F3000030F4009931882156
:103790009B316E302000A7002330A8007108270756
:1037A00086007208283D870001083F39A9000130D2
:1037B000A935FF3E031DD82B2935AA002A08FC0095
:1037C0007C08A50025082100DE000800F9008030F3
:1037D000A5002508F70079089D316C259B317908F3
:1037E0002000A500A6012508F1002608F2000930F6
:1037F000F3000030F400993188219B3171302000B2
:10380000A7002330A8007108270786007208283D0A
:10381000870001080339A9000130A935FF3E031DC7
:103820000D2C29350C39AA002A08FC007C177C08CD
:10383000A50025082100DE0008003F2C0D30890B73
:103840001F2C00005A2C1A30890B242C00325A2CC1
:103850002830890B292C5A2C3530890B2D2C00004F
:103860005A2C4230890B322C00325A2C5030890BA2
:10387000372C5A2C5D30890B3B2C00005A2C200031
:103880006A08003A03195A2C0A3A03191E2C1E3AE8
:103890000319232C0A3A0319282C363A03192C2C25
:1038A0001A3A0319312C0E3A0319362C7A3A0319B5
:1038B0003A2C5A2C983174200800F200F4012100AF
:1038C0000C16F3018C1520000C1E6A2C0130F1003F
:1038D0007108F4077435F1007108F40021008C11AF
:1038E0000130F1007108F30707307302031C622CEA
:1038F0008C1520000C1E812C0130F1007108F4079A
:10390000852C003200320032003221008C11720806
:1039100003190C12003200320032003221008C15E3
:103920000430890B912C21008C11003200320032BE
:10393000003221000C1674080800F800F70178081E
:10394000F5007508F6000230F5007508EB0021005F
:1039500069087802031CAE2CF801B22C0130F50086
:103960007508F8070530F5007508F10078089831FA
:10397000DE209C31223E8600023087000118D52CC3
:10398000210069087802031CC72CF801CB2C0130F8
:10399000F5007508F8070130F5007508F7070E30D7
:1039A0007702031CB22C2000EB0176087806031D79
:1039B000DC2C2000EB01EB0A780808000D30200019
:1039C000AA002A082100E900D8012000E201E40150
:1039D000E3012100CA019831C2209C31ED01ED0ABA
:1039E0002000E0010830AA002A082100EB00433043
:1039F0002000AA002A082100EA00E801E80AC6011E
:103A0000DD019F3117279C312000AB012B0893313A
:103A100004239C3120002B089B3115239C31063058
:103A200020002B020318192D2B08A03E86008701C9
:103A300081010130AA002A08AB070E302B020318BF
:103A40000800062DF9004030A5002508F700790888
:103A50009D316C259D3179082000A500A60125081F
:103A6000F1002608F2000930F3000030F40099312B
:103A700088219D3170302000A7002330A8007108F4
:103A8000270786007208283D87000108A900290839
:103A9000FA00B4307A02031C4F2DB4305A2D78301E
:103AA0007A02031C552D78305A2D3C307A02031CC3
:103AB0005B2D3C30FA027A08A5000130A535FF3EA7
:103AC000031D5E2D2535A6002608FC007C08A500F8
:103AD00025082100DE000800F8007808A000A101F8
:103AE0002008F1002108F2000930F3000030F40052
:103AF000993188219D3169302000A2002330A30034
:103B00007108220786007208233D870001083F39AB
:103B10007707A40024082100EF0078082000A00007
:103B2000A1012008F1002108F2000930F300003063
:103B3000F400993188219D3169302000A2002330A2
:103B4000A3007108220786007208233D8700011F29
:103B5000B12D21006F092000A00020082100EE00F7
:103B6000080021006F082000A00020082100EE00BE
:103B70000800F900F701F80122000C119931BF216A
:103B80009D31013A031DD32D2100E801E80A0130DF
:103B9000F7070030F83D0230780200300319770251
:103BA000031CBE2DE8017908F3000430F336890BBD
:103BB000D62D73080F39F4007408F60079080F3910
:103BC000F3007308F5007203031DE92D22008D1523
:103BD000EB2D22008D110D1098316C209D3176084F
:103BE000993157219D310C150D30890BF52D0000B1
:103BF00022000C117508993157219D310C150D309B
:103C0000890B002E000022000C119831682008005A
:103C1000F801F31F122EF209F309F20A0319F30A4D
:103C2000F801F80AF51F1D2EF409F509F40A031925
:103C3000F50A0130F6007608F806F901FA01720873
:103C4000730403194C2EF701F70AF31B312E0130D0
:103C5000F235F30D890B282E0130F6007608F707B0
:103C6000252E0130F935FA0D890B322E73087502B5
:103C7000031D3C2E72087402031C432E7208F402CA
:103C80007308F53B79140130F336F20C890B442E9E
:103C90000130F702031D312E78080319542EF9095B
:103CA000FA09F90A0319FA0A7A08F3007908F20006
:103CB0000800F9004030A5002508F70079089D317B
:103CC0006C259E3179082000A500A6012508F10089
:103CD0002608F2000930F3000030F4009931882101
:103CE0009E316D302000A7002330A80071082707FF
:103CF00086007208283D870001083F39A90001307D
:103D0000A935FF3E031D802E2935AA002A08FC0094
:103D10007908A500A6012508F1002608F20009305F
:103D2000F3000030F400993188219E316D3020007D
:103D3000A7002330A8007108270786007208283DD5
:103D40008700011FA92E7C09A50025082100DE009F
:103D500008007C08A50025082100DE0008002308D3
:103D6000FA002208F9009F3189279E3199311521E7
:103D70009E31200025080319E22E25087F3EFB0016
:103D80007B08A80002302406031DCB2E2808403EE5
:103D9000FB007B08A80003302406031DD42E28084E
:103DA000143EFB007B08A80004302406031DDD2E12
:103DB0002808543EFB007B08A800F20128089D312A
:103DC000B9259E31043020002602031CEE2EF2019C
:103DD000F20A210066089D31B9259E31033020008A
:103DE0002602031CFA2EF201F20A210065089D3119
:103DF000B9259E31023020002602031C062FF20155
:103E0000F20A210064089D31B9259E31F201F20ABF
:103E1000210063089D31B9259E3120002708031930
:103E20000800F201F20A27089D31B9250800083080
:103E300098319D209F315A3A031D252F0830983123
:103E40009D209F31013A031D862F5A30FB007B08CD
:103E5000F70008309931A3219F312930FB007B08FE
:103E6000F70001309931A3219F310230FB007B081C
:103E7000F70002309931A3219F31F70103309931C6
:103E8000A3219F311430FB007B08F70004309931E7
:103E9000A3219F314330FB007B08F70005309931A7
:103EA000A3219F313130FB007B08F7001530993199
:103EB000A3219F31F701F70A17309931A3219F31D0
:103EC000F701F70A18309931A3219F313C30FB00EC
:103ED0007B08F70014309931A3219F310430FB0097
:103EE0007B08F70016309931A3219F314B30FB003E
:103EF0007B08F70019309931A3219F313230FB0044
:103F00007B08F7001A309931A3219F319331A72301
:103F100008002100B401B501FF3079052000A000A0
:103F200007307A05A100E830F1000330F2002108E3
:103F3000F4002008F3009B3148239F3172082100D0
:103F4000B3007108B2003308F2003208F1001830F3
:103F5000F300FC30F400993188219F3120002008C3
:103F60007107A0002108723DA1006430F10000300B
:103F7000F2002108F4002008F3009B3148239F3110
:103F800072082100B1007108B0003108F200300859
:103F9000F1009C30F300FF30F400993188219F310B
:103FA000200020087107A0002108723DA1000A30FE
:103FB000F1000030F2002108F4002008F3009B31EA
:103FC00048239F3172082100AF007108AE002F080E
:103FD000F2002E08F100F630F300FF30F4009931C2
:103FE0008821200020087107A0002108723DA1004F
:103FF00021082100AD00200020082100AC000800AD
:020000040001F9
:04000E00E43FFF1FAD
:08000000FF3FFF3FFF3FFF3F00
:10E00000FF0029000200000014004300FF00FF0091
:10E010005A00FF00FF00FF00FF00FF00FF00FF00AD
:10E02000FF00FF00FF00FF003C0031000400000083
:10E0300000004B003200FF00FF00FF00FF00FF0068
:10E04000FF00FF00FF00FF00FF00FF00FF00FF00D8
:10E05000FF00FF00FF00FF00FF00FF00FF00FF00C8
:10E06000FF00FF00FF00FF00FF00FF00FF00FF00B8
:10E07000FF00FF00FF00FF00FF00FF00FF00FF00A8
:10E08000FF00FF00FF00FF00FF00FF00FF00FF0098
:10E09000FF00FF00FF00FF00FF00FF00FF00FF0088
:10E0A000FF00FF00FF00FF00FF00FF00FF00FF0078
:10E0B000FF00FF00FF00FF00FF00FF00FF00FF0068
:10E0C000FF00FF00FF00FF00FF00FF00FF00FF0058
:10E0D000FF00FF00FF00FF00FF00FF00FF00FF0048
:10E0E000FF00FF00FF00FF00FF00FF00FF00FF0038
:10E0F000FF00FF00FF00FF00FF00FF00FF00FF0028
:10E10000FF00FF00FF00FF00FF00FF00FF00FF0017
:10E11000FF00FF00FF00FF00FF00FF00FF00FF0007
:10E12000FF00FF00FF00FF00FF00FF00FF00FF00F7
:10E13000FF00FF00FF00FF00FF00FF00FF00FF00E7
:10E14000FF00FF00FF00FF00FF00FF00FF00FF00D7
:10E15000FF00FF00FF00FF00FF00FF00FF00FF00C7
:10E16000FF00FF00FF00FF00FF00FF00FF00FF00B7
:10E17000FF00FF00FF00FF00FF00FF00FF00FF00A7
:10E18000FF00FF00FF00FF00FF00FF00FF00FF0097
:10E19000FF00FF00FF00FF00FF00FF00FF00FF0087
:10E1A000FF00FF00FF00FF00FF00FF00FF00FF0077
:10E1B000FF00FF00FF00FF00FF00FF00FF00FF0067
:10E1C000FF00FF00FF00FF00FF00FF00FF00FF0057
:10E1D000FF00FF00FF00FF00FF00FF00FF00FF0047
:10E1E000FF00FF00FF00FF00FF00FF00FF00FF0037
:10E1F000FF00FF00FF00FF00FF00FF00FF00FF0027
:00000001FF
